:020000020000FC
:1000000013C012C011C002C00FC00EC01FB783952D
:100010001FBF18952FB72FBF18950FEF3FEF3A95D9
:10002000F1F70A95D9F70895F8DFF7DFF6DFF5DF86
:10003000F4DFF3DFF2DFF1DFF0DFEFDFEEDFEDDF44
:10004000ECDF32E039BF3327232F33BFBB9ABC9A92
:10005000C39AC49A30E438B944275527882731E039
:10006000732F789432E033BF8827002702BFB199FD
:10007000FECF33278827B19BFECF382F333090F344
:10008000882734E23A95F1F7332732BF32B73F3F42
:1000900060F7B199FBCF32B7002702BF393628F39A
:1000A0003B3910F461E005C03D3C10F462E001C052
:1000B00063E0222309F4262F213081F02230D9F089
:1000C000623011F4772723C0713009F1613019F0E3
:1000D00071E050951CC071E0409519C0613019F471
:1000E0004427552714C0623019F04FEF5FEF0FC05F
:1000F0004FEF55270CC0613019F44FEF552707C05B
:10010000623019F044275FEF02C04427552744238B
:1001100011F0C39801C0C39A552311F0C49801C0CF
:08012000C49AA5CF0000FECF38
:00000001FF
